:100000001CC081C180C17FC17EC17DC17CC17BC15B
:1000100007C179C178C177C176C175C174C173C197
:1000200072C171C170C16FC16EC16DC16CC16BC154
:100030006AC169C13F003F02800011241FBECFEF9B
:10004000CDBFDFE3DEBFE4E3F0E040E017C0B591F1
:10005000A59135912591059107FD0CC0959185914C
:10006000EF01F92FE82F05900D92A217B307D9F7EA
:10007000FE0104C01D92A217B307E1F7E933F407AC
:0A00800031F703D010C1F894FFCF50
:10008A00CF93DF93CDB7DEB7A097CDBFDEBFE0E059
:10009A00F4E080818068808380818F7B8083808187
:1000AA008F7D808380818F7E808364E074E0CE01BF
:1000BA00019677D0CE01019623D00F2EF2E8EF2ECB
:1000CA00F6E0FF2EF02D06E410E1EFD0FAD08BD047
:1000DA0004D1C7010197F1F7D7D00BD1682FCE0110
:1000EA00019639D0E8D0F3D07ED0FDD0C80101976F
:1000FA00F1F7CAD0FED0682FCE0101962CD0E5CFF9
:10010A00FC01A0E0B4E08C918E608C93A0E2B4E094
:10011A008C918F608C9384E094E08083918343E098
:10012A0042838483958352E056838087918761E076
:10013A00628724E234E0248735871686208B318B48
:10014A00628B248B358B568B208F318F428F848F15
:06015A00958F468F089509
:10016000EF92FF920F931F93CF93DF938C01C0E028
:10017000D0E0E62EF12CC7010C2E02C09595879594
:100180000A94E2F780FF03C0C80161D002C0C80131
:100190006FD021960C5F1F4FC830D10561F7DF91FA
:0C01A000CF911F910F91FF90EF900895F8
:1001AC00CF93DF93CDB7DEB7A097CDBFDEBF9C0159
:1001BC00FE01319690E092831382608371839F5F7E
:1001CC0034969830C1F780E2FE013196D901019046
:1001DC000D928A95E1F7C901A096CDBFDEBFDF91E4
:0401EC00CF91089512
:1001F0001092003F1092013F7894E0E0FAE081E035
:100200008287118281858E7F818788E290E086A334
:1002100097A3808186608083808181608083089538
:100220008F938FB78F939F93F8948091003F909115
:10023000013F01968093003F9093013F81E08093BE
:0E0240000B0A78949F918F918FBF8F91189524
:10024E00FC01A081B1818C9121E030E0028002C0DE
:10025E00220F331F0A94E2F7282B2C9381E083831D
:02026E000895F1
:10027000FC01A081B1818C9121E030E0028002C0BC
:10028000220F331F0A94E2F7209528232C93138220
:020290000895CF
:10029200F894E0E0FAE080818E7F808385818C6033
:0402A20085830895B3
:0E02A600EC0130D02ED0CE012ED0CE012DD0C6
:0C02B400E0E0F4E0808585FDFDCF0895BA
:0C02C000E0E0F4E0808584FDFDCF0895AF
:0C02CC00E0E0F4E0848180688483089501
:0C02D800E0E0F4E084818F7784830895D7
:0C02E400E0E0F4E0808586FFFDCF089587
:0C02F000E0E0F4E0808586FDFDCF08957D
:0A02FC008091003F9091013F0895AA
:020306007CCEAB
:02030800089556
:02030A00089554
:02030C00089552
:02030E00BBDE54
:00000001FF
